:030000000219FDE5
:03000B000200A848
:03002B000201646B
:03005B000202EEB0
:030073000202D4B2
:1000800002030406080C10182030406080040608A3
:100090000C10182030406080A0C000070F1F3F05E3
:1000A000050D050305030302C2AFC0D0C0E0206206
:1000B00017E5256002E473E525F4F58A758B00D217
:1000C00062D0E0D0D0D2AF3285268AC262E526F473
:1000D0006036306803207210758B00D0E0D0D0C23B
:1000E00090C291C292D2AF32C290C291C292206E9F
:1000F0000D20660A7401D5E0FDE57EF45290758B03
:1001000000D0E0D0D0D2AF32758A00C28DD2620169
:10011000FE01B7306805206602D29001B73068054D
:10012000206602D29101B7306805206602D29201A2
:10013000B7D29330680A2066077405D5E0FDD290E7
:1001400001B7D29430680A2066077405D5E0FDD265
:100150009101B7D29530680A2066077405D5E0FD95
:10016000D29201B7C2AFC2AD53E6EFC0D0C0E0D269
:10017000D3D2AFC2CEE52A6007207449152A21C523
:100180007800790020742EE580307E01F430E7029B
:1001900078FF53DACF207E0343DA20307E0343DA40
:1001A00010C2D8C271E580307E01F430E70279FFD9
:1001B000C3E89970CB306103752A18207403752A3F
:1001C00018885FD27020740DE52B6004152B21D5A3
:1001D00043DA01C2D82070024137A85F206102C211
:1001E00070207431C3E894F0400374F0F8E8C4540C
:1001F0000F28F87984B703024115C313C31387216D
:10020000200802C313200A06C3C898F8411528F82D
:10021000500374FFF8C3E895685003E568F8882236
:10022000E52D54066011E533C313C31324062522BC
:10023000F52250037522FF852224A824C3E52495C6
:10024000644002A8648825E5697002417BC3E8AA7E
:10025000699A5003E8FAE4F9EAC333FBE56BF45B0F
:1002600029400D256AF8E56A6002156A400B417B5A
:100270000AC3E56A9A5002056A78FF8826C26EC3EF
:10028000E52694F84002D26EC3E52594404002D2A0
:100290006420CF0AD0E0D0D043E610D2AD32C2CF36
:1002A000053A7801E52A6005307402152AC3E55F36
:1002B0009401400575620041CA756300756C00E5E4
:1002C000622401F56250037562FFD0E0D0D043E6AE
:1002D00010D2AD32C2AFC0D053E67FC2607591007C
:1002E000855694855795759104D0D0D2AF32C2AF60
:1002F00053E6EFC2ADC0D0C0E0C0F0D2D3D2AFA8B9
:10030000FBA9FCC2D8307102615553DACF207E03BD
:1003100043DA10307E0343DA20D271E580307E016B
:10032000F420E702612C88278928A17C53DACF20AA
:100330007E0343DA20307E0343DA10C2D8C2713024
:100340007402A1687800E580307E01F430E702A1F4
:1003500068885FA15053DACF207E0343DA20307ED5
:100360000343DA10C271206102812E53DACF207E5E
:100370000343DA10307E0343DA20C2D8D271885AA0
:10038000895BC3E89558F8E99559F97B007E087AAE
:1003900000C3E8948CE994005005755E00812088C4
:1003A0002178A2E6A8216055C3E894C8E9940050DA
:1003B00008E4D2E4FB7A0A61FBC3E89468E994019B
:1003C0005008E4D2E3FB7A0F61FBC3E894D0E994D0
:1003D000025008E4D2E2FB7A1E61FBC3E894A0E974
:1003E00094055008E4D2E1FB7A3C61FBC3E89498A1
:1003F000E994085008E4D2E0FB7A787E00C3E895DF
:100400005CFCE9955DFD30E70AECF42401FCEDF4B9
:100410003400FD755E00C3EC9AED9E5003755E01DD
:10042000885C895D855A58855B597802A150C3E87C
:100430009527F8E99528F9307C02A134307B02A198
:1004400034307A02A12D2075028151E9FDE8FC814A
:1004500070E9C313F9E813F8307902A12DE9C31349
:10046000F9E813F8307802A12DE9C313FDE813FC75
:0F047000206126C3EC941CED940240028187EDBD
:10047F007018C3EC94C850120529C3E529940A508B
:10048F0002A168755F00D270A168E5296002152985
:10049F007888E6F97400207F087896B90302789E71
:1004AF00E624FAFEE43400FFC3EC9EFCED9FFD92C0
:1004BF0008B90310A2085007207609D27681D330ED
:1004CF007602C276A2085016B9030DECF42401FC93
:1004DF00EDF43400FD0204ED78007900A134B90386
:1004EF0015EC33FCED33FDC3EC940AFCED9400FDE9
:1004FF0050047C007D00C3EC94FFED94004006781F
:10050F00FF7900A134EC8575F0A4C5F0A2F733F89C
:10051F007900400302055078FF7900020550E9C3C6
:10052F0013F9E813F8307C0EE9600278FFC3E81383
:10053F0038F8E43400F9C3E894FFE99400400278F6
:10054F00FF885FD270206102A168741FF4552F4B92
:10055F00F52FC274EB7002D274752A1830740375BC
:10056F002A0A306102A17C20740353DAFE2074033F
:10057F00752B06D0F0D0E0D0D0D2AD43E610327953
:10058F00010205AC79030205AC790A0205AC791EAC
:10059F000205AC79640205AC79C80205AC7817E4A2
:1005AF00D5E0FDD8FAD9F6227A147B780205D37AF2
:1005BF00107B8C0205D37A0D7BB40205D37A0B7BAB
:1005CF00C80205D37902B27DE4D294D5E0FDD29171
:1005DF00D5E0FDC291D5E0FDC294D5E0FDD290E506
:1005EF0076D5E0FDC2907496D5E0FDD9D9EAF8D55D
:1005FF00E0FDD8FBDBCED29422C37C007D0075F0EA
:10060F000005F0EA33FAEB33FB50F6EB13FBEA137A
:10061F00FAC3E9FFE8FEE89AF8E99BF95004EFF90D
:10062F00EEF8B3EC33FCED33FDD5F0DFEDF9ECF87C
:10063F0022E889F08A20D2D4F8A9F07B0030F70B9A
:10064F007BFFF42401F8E9F43400F9E88520F0A4E5
:10065F00ADF0F8E98520F0A4AFF0FEED2EF97400AF
:10066F003FFA7C04C3EA13FAE913F9E813F8DCF450
:10067F008BF030F70AE8F42401F8E9F43400F9E8D4
:10068F0089F0C2D4F8A9F02222C3E54113F9E5405D
:10069F0013F8C3E54598F8E54699F9500CC3E8946B
:1006AF0080E994FF40160206CFC3E8947FE99400D7
:1006BF0050030206CF787F79000206CF788079FF4A
:1006CF00884A894B22E54A2547F8E54B3548F98595
:1006DF004B20E4300701F43549FA30E709C3EA94B7
:1006EF00F0401502070DC3EA940F500302070D786F
:1006FF00FF79FF7A0F02070D780079007AF0C3E5D2
:10070F00249564500AC374019524500B02072BE5FE
:10071F004B20E70E02072BE54B30E7068847894849
:10072F008A492278A4E6FAC3E54A33F8E54B33F950
:10073F00D140E930E70BC3E89480E994FF4013E11F
:10074F0065C3E8947FE994005002E165787F7900F2
:10075F00E165788079FFE820E715C3E52398F84035
:10076F0009C3E89401400302078C780102078CE863
:10077F00F424012523F8400302078C78FF884C22CC
:10078F0078A5E6FAA848A949D140E930E70CC3E8B3
:10079F009401E994FF40160207C0C3E894FFE9945F
:1007AF000050030207C078FF79000207C078017973
:1007BF00FFE920E715C3E54C98F84009C3E8940119
:1007CF0040030207E778010207E7E8F42401254C0C
:1007DF00F840030207E778FF88242278FFC26420DD
:1007EF00693D206A12D264C3E541940A4009C3E50A
:1007FF002594405002C26479A1E76023E541601F50
:10080F0074FF8541F0848539F0306A0375F005A4D3
:10081F00F8C5F0600278FFC3E895675002A86788B3
:10082F006622C3E5409440E5419401E56650031408
:10083F000142046002F5662202084A2275E89022FE
:10084F007883E6FFE5E820ECF7A8BDA9BE0573C3E2
:10085F00E57394084052757300E9FA79A0E7604494
:0E086F00EA7007E574601B020885C3E8957403
:10087D006010E5745006600C140208910460F902D2
:10088D000891E574F574C394F6401B7564C0C39468
:10089D00064013756480C39406400B756440C39481
:1008AD0006400375640075BB0622E564F46002051D
:1008BD0064E573B4070375BB1022743279A687F013
:1008CD00A4C5F0A2F733F8C3E895644002A8648884
:1008DD00228824882588268867227540007541F076
:1008ED0022C2AF75C820A8CCA9CDAA3A30CF010A33
:1008FD0075C824D2AFAB3BAC3C883B893CC3E89B6D
:10090D00F8E99C206908F930670241032160AD3D8B
:10091D008A3DF9EA9DFA600478FF79FFAE3EAF3F5C
:10092D008B3E8C3FC3EC9FFCC3E99CF542A83BA9D1
:10093D003CC3E89EF8E99FF9C3E54113FBE540137D
:10094D00FAE82AF540E93BF54150067540FF75413F
:10095D00FF21AAAA40AB41AC40AD417E047F02C34A
:10096D00EB940440021E1FC3EB940840021E1FC3EC
:10097D00ED13FDEC13FCDEF7C3EA9CFAEB9DFBEFE8
:10098D006009C3E913F9E813F8DFF7EA28FAEB3940
:10099D00FB8A408B4150067BFF8B408B41C3EB9410
:1009AD00025002D2673069047F0321D57892E6FFA9
:1009BD00C3E537948240110FC3E53794A040010F72
:1009CD00C3EF940640027F057E04E541C4540FF940
:1009DD00E541C454F0F8E540C4540F28F8C3E89E2F
:1009ED00FAE99400FB4009C3EA9402EB9400500429
:1009FD007A02E4FB414FAA40AB41EBC4FEEAC4547A
:100A0D000F4EFCC3EA9CFAEB9400FBC3E813C3132F
:100A1D00F8EA28FAEB3400FB8A408B41C3EB9402D1
:100A2D004002C2677804EBC4FE7B00EAC4540F4E4B
:100A3D00FAC3EA98FA4005C3940250027A027892FA
:100A4D00E6FF306002414F855256855357D26043C1
:100A5D00E680C3E49AF8E49BF930670241E9E8FACD
:100A6D00E9FBD3E913FDE813FC88528953C3EF94D6
:100A7D00036038EF20E00DE82CF8E93DF9ECFAEDD4
:100A8D00FB020AA4E828F8E939F9C3E82402F8E9D9
:100A9D003400F97AFE7BFFC3EF9403400E8A548B2A
:100AAD0055884E894F8C508D51611D885489558ABA
:100ABD004E8B4F8C508D51306920C3E533940340DC
:100ACD0019E542A2E713F8E555F4240138400B204F
:100ADD00E7087554FFF42401F555611DE8FAD3E8D4
:100AED0013FC8852C3EF94036020EF20E007E82C3D
:100AFD00F8ECFA6109E8282402F87AFEC3EF9403B2
:100B0D0040088A54884E8C50611D88548A4E8C50F2
:100B1D00E56BC3335002646BF56B30600261277572
:100B2D003402D26043E680E52D54066026A840A924
:100B3D0041C3E913F9E813F8C2AF53E67F7591008D
:100B4D00C3E498F594E499F595759104D26043E664
:100B5D0080D2AF22D265754400752000306B0375CD
:100B6D002040020B80D265754400752040306B0328
:100B7D00752000D2AF7801206722E52D5406600262
:100B8D00C265C3E541940540137802940540087889
:100B9D0003940540027806306902780A206019E551
:100BAD0044601530690AC3E53394034003D5340618
:100BBD00D2AFD26C8152712FD2AF0000C2AF20677D
:100BCD0026E541C3FB940F40027B0FEB24053073E8
:100BDD000123306A02742820620123F930690279F9
:100BED0082E58BC39940B50544E59BF45440B5208F
:100BFD0002813C30690A08C3E8940A40010861A9E2
:100C0D002065026180C26553E67F759100306710E3
:100C1D007594007595FE759104D26043E6806180F0
:100C2D00AE40AF41C3E49EF594E49FF5958123C397
:100C3D00E5339402500261803065026180D80281F3
:100C4D005061A9C26C53E67F75910085549485550A
:100C5D0095759104854E56854F57D26043E680D2E7
:0F0C6D00AFE52D54066008206A020533020C8C97
:100C7C00306C0D206B0A2065071581158102150952
:100C8C002278003064053065027801E53775F0078D
:100C9C00A4F9E5F028F5F0E9A2F013A2F113A2F201
:100CAC0013F537C394785003753778C3E537953807
:100CBC004008D266C290C291C29230600281C68551
:100CCC005056855157D26043E68022207D11C2AF29
:100CDC00754302D294C293D2AF759F11020EA6C275
:100CEC00AF754302D294C295D2AF759F11020EA676
:100CFC00307243207D20C2AF754303900142757E54
:100D0C0010C292D295306204D291A11AC294D2AF81
:100D1C00759F01020EA6C2AF754303900142757E0A
:100D2C0010C290D293306204D291A13AC294D2AF45
:100D3C00759F21020EA6207D17C2AF75430390014B
:100D4C001DC292306202D291D2AF759F01020EA6E3
:100D5C00C2AF75430390011DC290306202D291D292
:100D6C00AF759F21020EA6207D11C2AF754304D230
:100D7C0093C295D2AF759F21020EA6C2AF754304E4
:100D8C00D295C293D2AF759F01020EA6307243204A
:100D9C007D20C2AF754305900131757E08C291D29A
:100DAC0094306204D290A1B6C293D2AF759F110257
:100DBC000EA6C2AF754305900153757E20C291D229
:100DCC0094306204D292A1D6C295D2AF759F110213
:100DDC000EA6207D17C2AF754305900113C291304A
:100DEC006202D290D2AF759F11020EA6C2AF7543AC
:100DFC0005900127C2913062EBD292D2AF759F1150
:100E0C00020EA6207D11C2AF754306D295C294D2B4
:100E1C00AF759F01020EA6C2AF754306D293C29462
:100E2C00D2AF759F21020EA6307242207D20C2AF38
:100E3C00754301900153757E20C290D293306204A9
:100E4C00D292C152C295D2AF759F21020EA6C2AFEB
:100E5C00754301900131757E08C292D295306204BF
:100E6C00D290C172C293D2AF759F01C1A6207D16DC
:100E7C00C2AF754301900127C290306202D292D268
:100E8C00AF759F21C1A6C2AF754301900113C292E9
:100E9C00306202D290D2AF759F01C26622900111CE
:100EAC00757E00C290C291C292D293D294D295C256
:100EBC006222788076FF0876FF0876FF0876FF08B6
:100ECC00760308760408760B087603087601087614
:100EDC0001788C76010876FF0876FF0876FF087695
:100EEC00FF0876FF0876030876FF0876FF0876FF82
:100EFC000876250876D00876FA0876FA087604087B
:100F0C0076FF08760108760008767A0876FF087670
:100F1C0001087601087600087603227887E6FFC27E
:100F2C0072BF0302D2727888E6C394036008C27D54
:100F3C00E630E102D27DC27E7889E630E102D27ED3
:100F4C00C3EF94026008758E01D273020F5F758E29
:100F5C0000C273227880E6149000809378A4F6780F
:100F6C0081E6149000809378A5F67886E6149000BC
:100F7C008D9378A6F6789CE67538FF75390CB4021B
:100F8C00067538A075390AB40306753882753905AB
:100F9C0078A3E61490009A93F569D1A92222789649
:100FAC00E6FA7897E6FB7888E6B40305C3EB940E73
:100FBC00FB307F047A007BFFC3EB9AFCC394825016
:100FCC00027C827575000575EC8575F0A4C3E5F09F
:100FDC00947D40F222D27FF1AA12059D7A007B000B
:100FEC007C10120593E55F2AFA74003BFBDCF37C62
:100FFC0004C3EB13FBEA13FADCF7FEC27F120FAA51
:10100C0022E5EF20E6037520000520903FFFE52048
:10101C00146006901DFF1460009304600375EF10BC
:10102C0053D9BF7581C043FF8012058E75EF004305
:10103C00B203E5B3240420E70DF521E5E320E00637
:10104C008521B343E301120EA97580FF75A40075C9
:10105C00F19075D47F75903875A53F75F23F75D5B5
:0F106C000075A60175E241E4F8F6D8FD756B0139
:10107B00120EBE12154B78988676753001C2AF12E0
:10108B0005A71205B712059D1205BE12059D120587
:10109B00C512059D1216641205A71205A71205A20B
:1010AB00C2AF78FA79FA308707D9FBD8F7021C0060
:1010BB00120F27120F60120FA9120FAA78988676BB
:1010CB00120EA975885075891275C824759104750F
:1010DB00D84075A82275B80275E690759B80759DF2
:1010EB000075D10775BC5875BB0675BA1175E880CC
:1010FB0012058ED2AF12084753DACF207E0343DAA4
:10110B0020307E0343DA1043DA01C2D8C2711205D4
:10111B00A7D2617B037A0CE55E70077A0CDB0302C6
:10112B0010AB12059D2070030210ABC270E55FC3BC
:10113B00940240E1E52F541F856160F561B560D5E0
:10114B00DAD5C26153DACF207E0343DA20307E0337
:10115B0043DA10C2D8C27178A2E67008D274E52FB8
:10116B0054E0F52FC2757529001205A2307409C31E
:10117B00E529940A4002D275120593780230740265
:10118B007800C3E55F9840F0C2AF1205B71205B700
:10119B001205B7D2AF1205A7754D007888E6B403D8
:1011AB0002418B120593788CE6C394015003021213
:1011BB008BE530C39401500302128B207435C3E5C9
:1011CB005F94FF500302128BC2AF1205CCD2AF1249
:1011DB0005A2C3E55F940150EFC2AF1205B712052C
:1011EB00981205B7D2AF1205A2C3E55F94FF40E991
:1011FB000216E97F05D27F120FAA1205A2C2AFC257
:10120B007F120FAAAE5FC3E55F947FD2AF407B1214
:10121B00058EC2AF1205CCD2AFDFDA120FE1C3EEEF
:10122B0094057897F61205A712158D12166C7F0A86
:10123B00D27F120FAA1205A2C2AFC27F120FAAAEA3
:10124B005FC3E55F947FD2AF50E412058EC2AF123D
:10125B0005B71205981205B7D2AFDFD4120FE1EE26
:10126B0024057896F61205A712158D12169B1205FA
:10127B00A2120FAAC3E55F94FF500221C60216E922
:10128B00C3E55F954D4003855F4D1205A27801794B
:10129B0088E7B403027805C3E55F98400221A6C234
:1012AB00AF1205CC1205CC1205CCD2AF1205A77527
:1012BB003000E4F531F5320531E531F470390532A2
:1012CB00789AE67819146012783214600D787D14D0
:1012DB00600878FA146003753200C3E53298401742
:1012EB0015327531B478998676C2AF1205CCD2AF70
:1012FB00789886761205A2120598E52A7005307447
:10130B000201AB78012074027806C3E55F9840A711
:10131B007888E6C3940360031205A2E52A700302E2
:10132B0010ABC2AF120EA9E4F522F523F524F52577
:10133B00F526F56AD2AF7885E6C333F568E4F54553
:10134B00F546F547F548F549F573F52CF52DF537C9
:10135B0075730875BB1012058E12084BE5E820EC6F
:10136B00FBA8BDA9BEE97001F8887412084F75730C
:10137B000875BB107887E6FE7602120F277887EE8A
:10138B00F6C2AF7564FF1208C78522648522658596
:10139B002266D2AF752201752401752501752601D0
:1013AB0085636C756D017888E6B40307C27D307672
:1013BB0002D27DD268D269753300120E0F120E3431
:1013CB001208E71208EE1208E71208EE1208E702FD
:1013DB0013EAC2AF120F27D2AF75730075BB06129B
:1013EB000B72120697120C8D120CD71208EE120B01
:1013FB0061306D031206982067031207EA3067030A
:10140B00120831120C8D120CFC1208EE120B7230FA
:10141B006D031206D4120C8D120D731208EE120B03
:10142B0061306D03120732120C8D120D981208EEFB
:10143B00120B72306D0312078F120C8D120E0F12DE
:10144B0008EE12084B120B61120C8D120E3412089F
:10145B004F1208EE306932206B2F85676485676504
:0E146B0085636C756D0179187A0CC3E53399B1
:10147900400CC269D26A8A357564FF021494C3E5C7
:101489005F940140030213EA021511306A1B206BB5
:1014990018E535147004C26A61DDF535C3E55F945A
:1014A9000140030213EA021511753600C3E562789B
:1014B90082985054307404E52A604D7888E6B40364
:1014C90017207D0520760781E130760281E1206BC6
:1014D90007D26B856764812978F0306B058567646D
:1014E9007820C3E54198500261EA306B1BC26BC298
:1014F9007D307602D27DD26A75351285676461EADC
:101509000536E55F6002A114753600C2AF120EA957
:101519007887E6FE7602120F277887EEF6E4F52241
:10152900F523F524F525F526F568C268D2AF12052D
:101539008E120EA9307409C3E5369405400201AB39
:1015490041BD901A0D78201215CFE520B45A0CA38D
:101559001215CFE520B4A50302156D120EBE1215A2
:101569008D02158C901A0378807B0A1215CFA30877
:10157900DBF9901A0F788C7B181215CFA308DBF9C9
:10158900901A2722C2AF12160E1215E8901A00748B
:101599000E1215D4A374041215D4A374141215D4FD
:1015A900901A0378807B0A1215D3A308DBF9901AE5
:1015B9000F788C7B181215D3A308DBF912162112A8
:1015C90015FF901A2722E493F622E6438F01538FE1
:1015D900FD75EF0275B7A575B7F1F0538FFE22437C
:1015E9008F02438F0175EF0275B7A575B7F1901A90
:1015F9000DF0538FFC22901A0D745AB1D4901A0E23
:1016090074A5B1D4227A3079D07820901A40B1CF1C
:10161900E520F709A3DAF7227A3079D0901A40E762
:10162900B1D409A3DAF922AB77A878BB010279848E
:10163900BB02027985BB03027986BB04027992BB9E
:1016490005027987BB060279A3BB0702799CBB080F
:10165900027988BB09027989E8F7227C051205A776
:10166900DCFB22C2AF1205B71205BE1205C5120571
:10167900CC1205981205B71205BE1205C51205CC84
:101689001205981205B71205BE1205C51205CCD26E
:10169900AF22C2AF1205CC1205C51205BE1205B79D
:1016A9001205981205CC1205C51205BE1205B7120E
:1016B90005981205CC1205C51205BE1205B7D2AFA1
:1016C90022AE77AF78C2AF1205B71205B71205B7C8
:1016D900120598DEF21205CC120598DFF8D2AF2276
:1016E900D16CD164D164757701757801757900D1B0
:1016F900CA7C05AD5F1205A7C3ED955F70F5C3E51B
:101709005F9401400AC3E55F94FF4032021725D177
:1017190030B18DD16CC2AF75EF10D164DCD50579CC
:10172900C3E5799403500280C6D1640578E577143E
:1017390090009F93F808C3E57898500280AED16471
:10174900D1640577C3E577940A5002809C120EBED6
:09175900B18DC2AF75EF10D1642F
:0319FD0002100DC8
:101A00000E0414FFFFFFFF03040B0301015AA5019D
:101A1000FFFFFFFFFF03FFFFFF25D0FAFA04FF01DE
:081A2000007AFF01010003FF41
:101A400023585033412320202020202020202020F4
:101A500023424C48454C4923463333302320202031
:101A60002020202020202020202020202020202076
:101C0000C2AFC2D353D9BF7581C043B20343FF8073
:101C1000752438752503B1C975EF0275E24043F1AB
:101C20008053A47F75D400D2877DFA780379E67C4F
:101C300010752200752300901DD67B0675249875BB
:101C400025013087028142208708D8FBD9F9DCF7CB
:101C500081B4308708D8FBD9F9DCF781B4B189E4C5
:101C600093A3C39A6004DDC381B4DBDBB17B600264
:101C7000812B7B08E493FAA3B15CDBF87A30B15C8A
:101C8000752200752300B17BEAFCEBFDC3ED94FEE9
:101C9000400EB17B8A278B28ED30E0048A828B834B
:101CA000B17B7AC270D8C3ED94FE601350CEBD00F4
:101CB00025EC60097520007521FF0200008100A855
:101CC00027A9280809D804D90281D3B17FEA89AAB3
:101CD000F281C50D81A0C3ED94035049EDA2E092BD
:101CE000007AC5C3E5829400E583941C50902000DF
:101CF00010438F02438F0175B7A575B7F1F030001F
:101D00001FA827A9280809438F01538FFDD804D99C
:101D100002A12089AAE275B7A575B7F1F0A3A10DBC
:101D2000538FFC817C7AC1BD030CE493A3FAB140CC
:101D3000DCF8B138817C817EAA22AB23B15CEBFA5E
:101D4000EA6222752608C3E52313F523E52213F57D
:101D50002250066323A0632201D526EAB1C9B1C986
:101D600075260AEAF4200102D287300102C287B147
:101D7000C9C3134002C201D526EB22B17FEAFB2082
:101D80008702A17F308702A184752608AE24AF2583
:101D9000C3EF13FFEE13FEB1CDB1C9C3EA13308711
:101DA000024480FA30E703632201C3E52313F523DD
:101DB000E52213F52250066323A0632201D526D91C
:101DC000E52265236523F52222AE24AF250E0FDE22
:101DD000FEDFFCD20122424C48656C693437316326
:041DE000F3300601D5
:00000001FF
